:020000040000FA
:0400040000EF08F011
:0600080001015DD91100A9
:10001800D8CF00F0E0CF01F0026E010116D80250EF
:0A00280001C0E0FF00C0D8FF100087
:100040000F013BEC22F0000102E3D8801200D890AF
:100050001200E9CF03F0EACF04F0FACF05F0FBCFAE
:1000600006F014AD3ED09DA03CD09EA03AD09E900C
:10007000CD900201F9504444F92603D00DD017D099
:1000800028D0010181A006D0452A090E456429D057
:10009000442A27D0456A25D0010181B022D06E0EB6
:1000A000436E02016D6B080E476E442A1AD0D89039
:1000B00081B0D8804636472E14D0020EEA6E43C077
:1000C000E9FF46C0EFFF6D2B432A080E476E442A16
:1000D00008D0010181B002D0440603D0446A456AC9
:1000E0002D8A010114AB63D09DA813D09EA811D016
:1000F0009D9813B105D012A503D012892D8009D087
:1001000002EE4BF00A51E926EFCFADFF13810A2B27
:1001100000079DAA4CD09EAA4AD0356A096AABA2B4
:1001200003D0AB98AB8837D0ABA409D0AE50010E4A
:10013000096E12A730D03B0EAF6E12972CD0040E72
:100140000201046F426AAECF07F0010107BE046BE3
:1001500002EE0BF00451E92607C0EFFF12A704D00E
:100160003B0EAF6E129712D013A110D002EE4BF0DF
:100170000951E926EFCF08F00750081803E0010EF7
:10018000096E04D0092B099B00679D88096603D07E
:100190002D82042B049B13A10AD0095208E013916D
:1001A0009D9812892D80630EAF6EAD6A12879DA255
:1001B00007D09EA205D09E92CA949E9C9D8CC2821E
:1001C0009DAC78D09EAC76D09E9C1C0EC214316F34
:1001D000D8903133D8903133C4CF08F0C3CF07F073
:1001E0000F0E086402D0076A086A01EE1DF0D8906D
:1001F0003135E92607C0EEFF08C0EEFF139D3151EF
:1002000009E0010A10E0030A17E0060A18E0020AF2
:1002100019E021D007502D5D08502E59D8A0138D1C
:10022000010E316F18D007502D5D08502E59D8A0FF
:10023000138D020E316F0FD0040E316F0CD0060EED
:10024000316F09D0A90E075C010E085802E2138B2A
:1002500001D0139B316B13AD21D089968998899C6D
:100260008BCF09F0FC0E09148B6E8FCF09F08C6ACE
:100270008D6A8ECF09F0030E09148E6EE00E0914FC
:100280008F6E1489336B020E0201056F0101138713
:10029000899E0201086F010113898A9AD89031372B
:1002A000D8903137318131C1C2FFF00ECC6E9E92B1
:1002B0009D82CA8405C0FAFF06C0FBFF03C0E9FFA8
:1002C00004C0EAFF120014AD09D0F2A807D0F2A2D0
:1002D00005D0F292CF68640ECE6ECD8014AB11D0F3
:1002E000F2A80FD0F2A20DD0F292F2981285356AE0
:1002F0002DB007D013B105D00D0E0F6102D0020E44
:040300000F271200B1
:1004000000011EDE03E30D01F4D90001000100EF3D
:1004100008F01200146A1350146009D09E90B10EB7
:10042000CF6ECD809EA0FED7CD90142AF4D71200B7
:10043000898E126A115012600AD0899E0A0E136EBC
:10044000E9DF898E280E136EE5DF122AF3D7C80E76
:10045000136EE0DFEDD70DEE10F001010351E92638
:10046000EFCF13F00DEE10F0E926EF6A032B400EEC
:100470000361036B13500D011200152C02D0176A93
:10048000000C14C018F0182A1850166201D0186A0F
:100490000D0EEA6E18501324E96EEFCF17F01750C7
:1004A000100A03E0FD0E176EFD0C186A0D0EEA6EC1
:1004B00014501324E96EEF50181A142A14501662BF
:1004C00001D0146A1704196E19521FE0150615BEE3
:1004D00002D0156602D0176A000C0D0EEA6E145099
:1004E0001324E96EEFAE03D0FE0E176EFE0C0D0E58
:1004F000EA6E14501324E96EEF50181A142A14509F
:10050000166201D0146A1906DFD7183C02D01750C2
:1005100012001768FF0C9EAA14D0ABA203D0AB98B0
:10052000AB880FD0ABA402D0AE500BD0899E0DEE9D
:1005300010F00251E926AECFEFFF022B400E026110
:10054000026B0351025D116E11AE02D0400E1126F6
:1005500011522BE00DEE10F00351E926E50EEF628B
:1005600022D0100E136E03C114F011C015F0400E0E
:10057000166E83DF17C091FD0D01915107E0FD0A52
:1005800007E0030A05E0010A06E008D001010DD0EA
:1005900062DF01010AD012680101FF0C898E010E91
:1005A000126E0101010C57DF0101126A000C7FB2CB
:1005B000FED711C062FF12C063FF7F9E7F9C7F80C9
:1005C00061501200020E1D6E7F9E7F9C7F8418C0BA
:1005D00062FF19C063FF0DEE00F01BC01CF0EFCFEF
:1005E00061FF550E7E6EAA0E7E6E7F827FB2FED7B1
:1005F0007F806150EF6209D0020E1D6EEE50622ABC
:100600006250D8B4632A1E8002D01E9002D01C2EE5
:10061000E6D71EA002D0D88012001D2EE0D7D890B9
:100620001200899E020E256E7F8E7F9C7F847F8EB6
:1006300020C0F6FF21C0F7FF22C0F8FF7F88550ECB
:100640007E6EAA0E7E6E7F827F980A000DEE50F0BD
:1006500023C024F0EECFF5FF0F00242EFBD7550E5C
:100660007E6EAA0E7E6E7F827F9420C0F6FF0DEE16
:1006700050F0268023C024F00900F550EE1802E067
:10068000269002D0242EF8D726A004D09281898EFD
:10069000D8801200252ECAD7D89012007F8E7F9C5A
:1006A0002250F86E2150F76EC00E2014F66E0DEE3B
:1006B00050F0400E236E0900F5CFEEFF232EFBD73E
:1006C00012003F0E18141F6E500E1F241D6E1D06C3
:1006D0001E6A1F6A1B501F5C1F501B18D8B0800A6F
:1006E00036E61D2A900E1D6219D0500E1D6E93CD58
:1006F00020F094CD21F0226A400E236E92DF0CE3AD
:10070000400E9327000E942393CD20F094CD21F03A
:10071000226AC4DF929102D0D89012000D0EEA6EC8
:100720001EC0E9FFEFCF1CF019501A1003E1030EB1
:10073000186406D00D0EEA6E1DC0E9FF1CC0EFFF65
:100740001E2A182A000E19221A221F2AC3D7D8805F
:1007500012001350176E1250166EC00E1114156E43
:10076000898E175003E1030E166407D0175005E178
:10077000010E155C0A0E16582EE317502CE1F00EF0
:10078000166029D092A10BD015C093FD16C094FD20
:1007900093CD20F094CD21F0226A80DF9291155004
:1007A00093630ED0165094630BD0176609D011C016
:1007B00018F012C019F013C01AF014C01BF081D742
:1007C00093CD20F094CD21F0226A400E236E29DFD4
:1007D000C7E2D8901200F00E136209D011C018F0D1
:1007E00012C019F013C01AF014C01BF0EBD6D88059
:1007F000120092811092899E108001018CDEFF0A06
:100800000D0103E0FE0A07E0C5D010A2C3D0040E1C
:10081000116E0EDEBFD0899E1EDE1DDE100AD8A42A
:10082000B9D019DE7F0AD8A4B5D015DE7F0AD8A4C6
:10083000B1D011DE7F0AD8A4ADD00DDE0A6E040E51
:10084000010103250C6E3F0E0C6402D0400E0C5EBD
:100850000DEE10F00C50E926F00EEF140D0108E03B
:10086000100A47E0300A55E0600AD8B484D092D02C
:10087000F2DD570A03E0010E116EDADDECDD1C0A31
:1008800003E0010E116ED4DDE6DD906F909F0AB497
:10089000908F020E010103250C6E3F0E0C6402D0F6
:1008A000400E0C5E0DEE10F00C50E926EFCF0BF071
:1008B0000D010BA00DD00BB206D0904D09D0020E49
:1008C000116EB6DD05D0906703D0020E116EB0DD5B
:1008D000C2DD906F909F0AB6908F0BA408D0116A6A
:1008E000126A65DE906103D0030E116EA1DD1082E5
:1008F00051D0B1DD0F6E0F9E0AB00F8EACDD0E6EC3
:100900000E9E0AB20E8EA7DD0D6E0D9E0AB40D8EE0
:1009100041D01DEE00F00C6A040E0C6009D09BDD86
:10092000E76E0A32D8A0E69ED8B0E68E0C2AF4D73D
:1009300092DD0B6E0C6A040E0C6009D08CDDE76E44
:100940000B32D8A0E69ED8B0E68E0C2AF4D70DC0A4
:1009500011F00EC012F00FC013F0080E146EF9DE85
:1009600006E3080E0D26000E0E220F2213D0050EF0
:10097000116E5EDD0FD092B10CD093CD20F094CDEE
:1009800021F0226A400E236E4CDE03E2050E116E4A
:100990004FDD109010B031D7120052BE09D0D6CF23
:1009A0000AF055500A5C565E0AC055F0D8A0528E27
:1009B0001200D6CF0AF053500A5C545E0AC053F0BE
:1009C000D8B012007D0E5426050E0B6E010E0C6E73
:1009D00000EE48F052500C140DE1EF06EF3C03D04E
:1009E000EE50EF06ED50EF50EE50EF1002E10C50DC
:1009F0005212ED50020EE926000EEA22D8900C3673
:060A00000B2EE8D71200E6
:10100000010103D000EC02F001010D0192B303D005
:1010100020EC00F00D010101BCEC22F022EC23F0E9
:101020007CEC23F05268536A546AC60ED56E2D6A62
:101030000101C4EC23F02D862D88D08EF28EF28C27
:101040002E6A2F6A306A316A800E416E426E376EA8
:10105000386E3C6E3D6E3E6E3F6E406E356E326E4B
:10106000336E346E366E3B6E396E3A6E336A346A66
:10107000366A386A3B6A396A3A6A0400D19014AD1C
:1010800003D0326AF292F2889E9C9D8C030EC26E4F
:1010900084DC8FDC2EBE02D06AD82E6E2FBE02D02A
:1010A0007CD82F6E30BE04D002011AD9306E0101F7
:1010B00031BE02D0A7D9316E32BE02D0E8D9326E2D
:1010C00033BE02D0ADDA336E34BE02D045DB346EAF
:1010D00035BE02D065DA356E36BE02D0CFDA366E56
:1010E00037BE02D084DB376E38BE02D09BDB386E51
:1010F00039BE05D000018FEC15F0396E01013ABE02
:1011000003D080EC19F03A6E3BBE03D0EFEC12F046
:101110003B6E3CBE05D0000123EC18F03C6E010193
:101120003DBE05D0000161EC16F03D6E01013EBEF2
:1011300005D00001E9EC16F03E6E01013FBE05D07E
:10114000000141EC1DF03F6E010140BE05D00001E1
:1011500028EC1FF0406E010141BE03D096EC10F068
:10116000416E42BE95D79FEC10F0426E91D7F95078
:101170002E44F92601D004D0010E486E496A5290DF
:1011800052A0010CDC0E215D050E225903E27DEC1C
:1011900012F00101000C0101800CF9502F44F926D6
:1011A00001D004D00A0E4A6E4B6A529252A2010C30
:1011B00003019DEC1CF00F6A0101020E0F603DD08F
:1011C00003EE00F00F50E926EFCF0CF003EE02F033
:1011D000E9260C50EF140E6E03EE08F00F50E926CE
:1011E0000C50EF140B6E0E500B180D6E010E0A6EA4
:1011F0000A521BE003EE0AF00F50E926EF500D14DF
:101200000C6E0A500C160EE003EE08F00F50E926A3
:101210000A50EF1A14B506D003EE10F00F50E9266D
:101220000A50EF12D8900A36E3D703EE0AF00F50B7
:10123000E9260DC0EFFF0F2AC0D713A706D0020181
:10124000052F03D001011397898E010113A906D040
:101250000201082F03D0010113998A8A010113BDED
:1012600002D0325307E0322B050E326504D0326BC8
:101270003A6A01D03A6A3C6A406A3D6A3E6A14ABF7
:1012800022D081B008D012AF0DD00D2B0A0E0D6305
:1012900009D0129F07D00D6B12BF04D00E6702D089
:1012A000010E0E6F0E530FE00E2B180E0E650BD0B5
:1012B0000E6BF29EF292F288AB889E9A9D8A9D9860
:1012C000AC8AF28E128F13BD08D014A906D0332B2E
:1012D0000F0E336502D0336B1499000C0101800CA2
:1012E0000101F9503044F92601D008D0640E4C6E4B
:1012F0004D6A5294020152B403D0010C0201FBD793
:1013000025C10AF026C10BF0D10E0A5C070E0B585E
:1013100015E3B80E0A5C0B0E0B5810E2010114B372
:1013200019D0070109A303D00101148102D00101E2
:10133000149107010983010114830CD0010114A346
:1013400009D014A103D00701098302D00701099332
:101350000101149301011169020106530EE0060711
:101360000F0E06150AE1063B06070F0E061504E0F0
:10137000050E036F416A068B063B075307E0072FF4
:1013800005D0050E036F416A010E076F0A5307E08F
:101390000A2F05D0050E046F426A010E0A6F010183
:1013A00014AF09D013B707D0050E0201036F010E69
:1013B000076F416A010112AB21D00D800C6A020E49
:1013C00002010C6017D003EE10F00C50E926EF502C
:1013D000D8A40D9003EE18F00C50E926EF50D8A4D5
:1013E0000D9003EE1AF00C50E926EF50D8A40D90A2
:1013F0000C2AE5D70DA002D00101129B0201000CBE
:101400000201800CF9503144F92601D005D0E80ED4
:101410004E6E030E4F6E529652A6010C147713AB0C
:1014200014D013BD12D013B907D014A705D0640E81
:101430000201036F416A010113B707D014B705D049
:10144000640E0201046F426A010112AD1CD0128BBE
:1014500003EE00F01051E926EFCF0AF003EE10F092
:10146000E9260A50EF1203EE00F01051E926EF1CB6
:101470000A6E03EE10F01051E9260A50EF12102BFD
:10148000020E1061129D1495000C0101800CF950A0
:101490003244F92600D02DAA010C22EE6DF002EEA6
:1014A00079F01F0EDF14406F4029DECFEEFFE80613
:1014B000000AFBE12D9A436B010E416F40514161DF
:1014C00008D002EE79F04151E926EF50431B412B41
:1014D000F5D702EE79F04151E9264351EF625CD035
:1014E0007AC245F1454958D002017AAF30D0050E95
:1014F000010140612CD002017BAF4ED03F0E7A1526
:10150000040DF3CF45F1070E7B15D890E8300101AB
:101510004513040E455F02017B1D700BE83A0F0B6B
:101520000101466F010E02017B15E83AF00B010143
:10153000426F46134551116302D046532DE045C119
:1015400011F145C115F146C116F1000E8DDA020107
:101550007AAF22D0040E010140651ED03F0E020179
:101560007A150101466F7BC245F1455102016B635B
:1015700005D00101465102016C1908E00F0E01016E
:1015800045630AD0270E466307D00201EC0E7C1596
:10159000EC0AD8B4F4EC20F00101000C0101800C3D
:1015A000F9503544F92602D007D035D01285D6CF70
:1015B00055F0960E566E529E52AE010CF292F28883
:1015C0000F450A6E0A44060FF924D8B0FA2AF96EBC
:1015D000960E1DD08E0E1BD0860E19D07F0E17D002
:1015E000780E15D0700E13D0690E11D0610E0FD089
:1015F0005A0E0DD0520E0BD04A0E09D0430E07D012
:101600003C0E05D0340E03D02D0E01D0000ED6CFE7
:1016100055F0566E529E52AE020C12950101800C8E
:101620000201F9503344F92600D001012DA2010C2A
:1016300002010BAF1ED048D90A6E0A50010119E011
:10164000FF0A05E102010B6B0101139112D012EEAA
:101650000BF004EE00F00251E926E6CFEEFFE95070
:10166000D8B404EE00F00A2EF8D7E9CF02F11391B6
:101670002D802D920101000C0101800C3650D8A460
:10168000800C0251031965E004EE00F00351E926D5
:10169000EFAE5ED004EE00F0E926EF50830A0DE0D5
:1016A000330A0FE0010A22E0030A2FE05F0A3CE060
:1016B000020A47E05B0A4AE04BD00701B3EC10F0A6
:1016C00047D03BEC10F00AC015F10BC016F11551D4
:1016D0001615FF0A3DE0000EC7D912C00AF013C06C
:1016E0000BF06AEC14F0139F3F6A32D03BEC10F021
:1016F0000AC015F10BC016F115511615FF0A28E0A6
:10170000010EB2D9139F3F6A23D03BEC10F00AC000
:1017100015F10BC016F115511615FF0A19E0020E4E
:10172000A3D9139F3F6A14D0DCEC0FF00AC015F167
:101730000BC016F115511615FF0A0AE0138F3F6A08
:1017400007D007018FEC1FF0010102D0F3EC21F06C
:10175000032B000C0101800C0201F9503444F926DE
:1017600003D002D02ED038D001012DA4010C2D942D
:1017700002014B390F0B01010F6F0F0E02014B15C8
:101780000101006F010E096F0A6F14AD15D0040E30
:10179000046F576A005157600DD002EE4CF057505D
:1017A000E926EFCF58F002EE0BF0E92658C0EFFF24
:1017B000572AF0D72D8217D012B502D012BF03D00E
:1017C000020C0101F9D7E0EC23F012B5D6D79D88C1
:1017D0002D902DB003D0030C0101FBD712A902D02C
:1017E0001299CBD70F6B2D86000C0101800CF9509C
:1017F0003744F92600D02DA6010C2D9612EE2BF0C1
:10180000E6CF0AF022EE4BF00AC0DEFF0A060B6AB2
:10181000E6CFDFFFDE500B1A0A2EFAD70B1CDF6E65
:101820002D84800CF9503844F92601D006D0075198
:10183000056303D00851061944E02DA6010C2D962E
:1018400022EE4BF00551E96E050E0625EA6EEFCF4C
:101850000AF00AC0DEFF052B000E0623056705D03F
:10186000020E066302D0056B066B0A060B6A055171
:10187000E96E050E0625EA6EEFCFDFFFDE500B1A8C
:10188000052B000E0623056705D0020E066302D065
:10189000056B066B0A2EEBD70B1CDF6E0551075D3F
:1018A0000A6E065108590B6E0BAE02D0020E0B26C3
:1018B0000BBE05D0D00E0A5C010E0B58D8A02D88A7
:1018C0002D84000C0101800C0BAD14D00BAB0FD09C
:1018D000020E0101046101D0000C0CC20BF0030EDA
:1018E00002010B6403D0100E0B640BD0FF0C060E2C
:1018F0000B6E07D00BAB03D0040E0B6E02D0020EA2
:101900000B6E010104510B6212D00C6A0D6A02EEDB
:101910000BF00D50E926EF500C1A0D2A0B500D5C00
:10192000F6E30C28020102E10B501200FF0C000C40
:10193000176E1438030B186E1B9216BE1B821B9475
:1019400016B81B8401011BB013D01BA211D017A025
:101950000FD00F0E16141D6E15501C6E1C06000EB7
:101960001D5A1CC015F01DC016F016981BB4168821
:101970001F0E16161BB019D0185005E0010A06E01C
:10198000030A0AE011D01686169A31D0169A1686E6
:1019900016A82DD016962BD016341632153216985E
:1019A000D8B01688168A23D01200185005E0010A14
:1019B00009E0030A10E01AD01686100E14BC161A9D
:1019C000169A15D0169A100E14BC161A168616A85A
:1019D0000ED016960CD01634163215321698D8B092
:1019E0001688168A080E14BC161A01D01200D89058
:1019F00015361636D89015320751E96E050E0825B2
:101A0000EA6E040EEF6EA4DB0751E96E050E0825A1
:101A1000EA6EB00E1810EF6E9BDB0751E96E050EF3
:101A20000825EA6E15C0EFFF93DB0751E96E050E3E
:101A30000825EA6E16C0EFFF8BDB0551075D196EB6
:101A4000065108591A6E1AAE02D0020E1A261ABE94
:101A500006D0E10E195C010E1A58D8B02D98050E6B
:101A60000201036F416A12000A6E0F0E1615136E03
:101A70001551126E0F6A020E02010F60DAD10E6864
:101A8000010E106E1052D8B4D2D10E2A03EE00F01F
:101A90000F50E926EF1C1014D8B4C6D10F50400DDA
:101AA000F3CFD9FFF4CFDAFF100ED926070EDA22D2
:101AB000080E0E02F350D926000EDA220EA015D021
:101AC000080ED95E000EDA5ADCCF0BF0DD501C9404
:101AD0000BBC1C841C960BBE1C861CA602D01CA42E
:101AE00004D0080ED926000EDA22DECF14F0070E3D
:101AF000DF14156ED9CF1AF0DACF1BF0030ED926FA
:101B0000000EDA22DECF16F0DFCF1DF00F0EDE144E
:101B1000176EDECF18F0DFCF1EF00F0EDE14196E39
:101B20001AC0D9FF1BC0DAFFDECF0BF01C940BBC30
:101B30001C841C960BBE1C86DFCF0CF0DCCF1FF084
:101B4000DD501F38070B1F6E0B38030B0A6256D08F
:101B50001250146253D01350156250D0030E0C145F
:101B60004DE01C92010116B91C82020EDFBE1C1A48
:101B70001F50040A03E0060E1F6209D002011CB2C6
:101B800003D01050A51302D0101CA5171C82020E02
:101B900002010A620ED00AC020F0299029921CB2DC
:101BA00029820EC021F00FC022F01050A4EC14F0D6
:101BB00025D01CB414D01CA612D00EA010D00AC080
:101BC00020F029901CB4298029821CB229920EC0D1
:101BD00021F00FC022F01050A4EC14F00FD00AC076
:101BE00020F029901CB4298029921CB229820EC0B1
:101BF00021F00FC022F01050A4EC14F0030ED926EF
:101C0000000EDA22DFCF0DF0D8900C32D8900C32D3
:101C1000030E0C147EE01C92010116B91C82030E07
:101C20000C14010A05E0030A07E0010A09E00AD0E2
:101C300002011CB209D06DD002011CA205D069D0EE
:101C4000020102D0020165D00DAE3DD012501662E5
:101C500060D0135017625DD0020E0DBC1C1A1F50CD
:101C6000040A03E0060E1F6208D01CB203D0105015
:101C7000A51302D0101CA5171C821CB414D01CA6DE
:101C800012D00EA010D00AC020F029901CB42980D8
:101C900029821CB229920EC021F00FC022F01050F0
:101CA000A4EC14F036D00AC020F029901CB429808E
:101CB00029921CB229820EC021F00FC022F01050D0
:101CC000A4EC14F026D01250146203D0135015184F
:101CD00008E0125018621DD0135019621AD01EAEBF
:101CE00018D002EEA8F00F50E926EFCF11F01CA299
:101CF00003D01050111202D0101C111602EEA8F0E1
:101D00000F50E92611C0EFFF03EE18F0E92610503E
:101D1000EF12020ED926000EDA22DFCF0DF0D89096
:101D20000C32D8900C32030E0C147EE01C92010190
:101D300016B91C82030E0C14010A05E0030A07E021
:101D4000010A09E00AD002011CB209D06DD00201DB
:101D50001CA205D069D0020102D0020165D00DAEEF
:101D60003DD01250186260D0135019625DD0020E3F
:101D70000DBC1C1A1F50040A03E0060E1F6208D097
:101D80001CB203D01050A51302D0101CA5171C8242
:101D90001CB414D01CA612D00EA010D00AC020F083
:101DA00029901CB4298029821CB229920EC021F0EE
:101DB0000FC022F01050A4EC14F036D00AC020F06E
:101DC00029901CB4298029921CB229820EC021F0CE
:101DD0000FC022F01050A4EC14F026D01250146260
:101DE00003D01350151808E0125016621DD013507E
:101DF00017621AD01DAE18D002EEAAF00F50E926D5
:101E0000EFCF11F01CA203D01050111202D0101C01
:101E1000111602EEAAF00F50E92611C0EFFF03EEF3
:101E20001AF0E9261050EF12D89010362BD60F2A50
:101E300022D61250010112000751E96E050E082545
:101E4000EA6E0B0EEF6E84D90751E96E050E082578
:101E5000EA6EED0EEF6E7CD90751E96E050E08258E
:101E6000EA6E0B0EEF6E74D90751E96E050E082568
:101E7000EA6E7F0EEF6E6CD90751E96E050E0825EC
:101E8000EA6E310EEF6E64D91438E8441F0B156EFC
:101E9000143A1442F80E1416030E13141412D890A8
:101EA0001436700E141A1480149ED8901332D890E1
:101EB00013320751E96E050E0825EA6E010EEF6E2A
:101EC00047D90751E96E050E0825EA6E13C0EFFFEA
:101ED0003FD90751E96E050E0825EA6E14C0EFFFE1
:101EE00037D90751E96E050E0825EA6E15C0EFFFD8
:101EF0002FD90751E96E050E0825EA6EEF6A28D939
:101F00000751E96E050E0825EA6EEF6A21D90551E1
:101F1000075D156E06510859166E16AE02D0020EF8
:101F2000162616BE06D0E10E155C010E1658D8B066
:101F30002D98050E0201036F416A1200136E14689A
:101F4000010113AF1AD01038E8461F0B1F0B176E94
:101F50001238E8461F0B1F0B186E070E10161216CC
:101F60000F50116227D01050126224D0146A1750FB
:101F7000186220D0010E146E1DD01038030B176E9E
:101F80001238E840E8423F0B030B186E17501862F6
:101F900011D00F0E10161214166E1150156E0F5030
:101FA000156208D01050166205D0146A12B8142AAF
:101FB0001350141A14501200032B04EE00F00351B6
:101FC000E926EF500B0A03E00A680B68FF0C032BAD
:101FD00004EE00F00351E926EF507F0A03E00A689F
:101FE0000B68FF0C032B04EE00F00351E926EF38D9
:101FF000070B030A03E00A680B68FF0C032B04EECF
:1020000000F00351E926070EEF14010A03E00A6805
:102010000B68FF0C032B04EE00F00351E926EFCF11
:102020000AF00AAC03D00A680B68FF0CD8900A3695
:10203000D8900A36032B04EE00F00351E926EFCFC7
:102040000BF0700E0B1AD8900B32030E0B140A1201
:102050000B3A0B461F0E0B16032B04EE00F0035138
:10206000E926EFCF0CF00C3A0C42F80E0C160C508F
:102070000B120A50120004EE00F00351E926EFCFD4
:102080000CF0032B04EE00F00351E926D890EF3456
:102090000A6E032B04EE00F00351E926EFCF0DF09A
:1020A00004EE00F0E9263F0EEF140B6E0E900DBC0F
:1020B0000E80030E0C14020A05E0030A0DE0010A6B
:1020C0001EE032D00EB003D00A680B68FF0C0A90F5
:1020D0000DBA0A800B8E28D00EB00BD00DBA02D0EC
:1020E0000DA804D00DAA05D00DA803D00A680B686E
:1020F000FF0CD8900B320A320B960B8C15D00EA029
:1021000003D00A680B68FF0CD8900B320A320BB66A
:102110000AD00AC00FF00BC010F007012BD80A68D4
:102120000B680101FF0C0B960A5012004150D8A415
:10213000800C03C205F21387899E0101800C425076
:10214000D8A4800C04C208F213898A9A0101800C79
:10215000072B000E0823076705D0020E086302D084
:10216000076B086B120009A503D00101106B128DDB
:1021700001011200070E1014166E0F50156EF80EA6
:10218000155C030E1658D8A0D2D0FC0E155C030EB9
:102190001658D8B0CCD0030E0F14146E10B8148497
:1021A000116A020E1160BED01268010E136E135236
:1021B000D8B4B6D0122A1150400DF3CFD9FFF4CFC6
:1021C000DAFF100ED926070EDA22080E1202F3509B
:1021D000D926000EDA22DECF17F0DF38030B196E96
:1021E0000F0EDE14186E18BC98D0030E1C6ED8901B
:1021F000183217321C2EFBD7186A070E1716DECFBF
:102200001AF01B901ABC1B80030E1A141BE0175007
:10221000146218D009A70AD01BA008D0195206E0F2
:1022200003EE10F01150E9261350EF1209A90AD05D
:102230001BB008D0196606D003EE10F01150E92645
:102240001350EF12DE50DECF17F0DF380F0B196E90
:102250001B9019B61B80030E19160F0EDE14186E94
:10226000030E1C6ED890183217321C2EFBD7186A3A
:10227000070E17160C0E1A141BE01750146218D014
:1022800009A70AD01BB008D0195206E003EE18F0D7
:102290001150E9261350EF1209A90AD01BA008D04B
:1022A000196606D003EE18F01150E9261350EF120C
:1022B000DECF17F0DF380F0B196E1B9019B61B809D
:1022C000030E19160F0EDF14186E030E1C6ED89035
:1022D000183217321C2EFBD7186A070E1716300E4D
:1022E0001A141BE01750146218D009A70AD01BB0AB
:1022F00008D0195206E003EE1AF01150E9261350E7
:10230000EF1209A90AD01BA008D0196606D003EE67
:102310001AF01150E9261350EF12D890133647D710
:10232000112A3FD7180E091502E00101128B07018F
:1023300012001B6E030EEA6E1AC0E9FF1B461B4615
:10234000F9501B44F926EF6A000E00003BD00A0E3C
:10235000EF6E000E37D0140EEF6E000E33D0230E4A
:10236000EF6E000E2FD0320EEF6E000E2BD0410E0E
:10237000EF6E000E27D0500EEF6E000E23D0640ECD
:10238000EF6E000E1FD07D0EEF6E000E1BD0960E6E
:10239000EF6E000E17D0C80EEF6E000E13D02C0E8D
:1023A000EF6E010E0FD0900EEF6E010E0BD0F40EFB
:1023B000EF6E010E07D0580EEF6E020E03D0200E06
:1023C000EF6E030EEC6E12001B6E030EEA6E1AC067
:1023D000E9FF1B461B461B44060FF924D8B0FA2A16
:1023E000F96EE80EEF6E030E3BD0DC0EEF6E050EBD
:1023F00037D0D00EEF6E070E33D0B80EEF6E0B0E47
:102400002FD0A00EEF6E0F0E2BD0880EEF6E130E96
:1024100027D0700EEF6E170E23D0280EEF6E230E0E
:102420001FD0E00EEF6E2E0E1BD0500EEF6E460E3C
:1024300017D0C00EEF6E5D0E13D0300EEF6E750E1E
:102440000FD0A00EEF6E8C0E0BD0100EEF6EA40E00
:1024500007D0800EEF6EBB0E03D0600EEF6EEA0E5B
:10246000EC6E12001B6E030EEA6E1AC0E9FF1B46EB
:102470001B46F9501B44F926050EEF6E000E3BD0AB
:102480000A0EEF6E000E37D0140EEF6E000E33D032
:10249000230EEF6E000E2FD0320EEF6E000E2BD0FB
:1024A000410EEF6E000E27D0500EEF6E000E23D0BF
:1024B000640EEF6E000E1FD07D0EEF6E000E1BD06F
:1024C000960EEF6E000E17D0C80EEF6E000E13D0F2
:1024D0002C0EEF6E010E0FD0900EEF6E010E0BD092
:1024E000F40EEF6E010E07D0580EEF6E020E03D001
:1024F000200EEF6E030EEC6E120013B548D00701EC
:1025000009A145D0F29E800E896E200E8A6E8B6ADC
:102510008C6A8D6A8E6A8F6A900E0A6E010E0B6E3F
:102520000AC012F00BC013F0030108510BEC22F0AB
:102530000A2A000E0B220AC012F00BC013F007513A
:102540000BEC22F0020E0A26000E0B220201002BD9
:10255000012302230AC012F00BC013F000510BEC50
:1025600022F00A2A000E0B220AC012F00BC013F050
:1025700001510BEC22F00A2A000E0B220AC012F0C5
:102580000BC013F002510BEC22F0010113850B0E6E
:10259000C26E0201C2B2FED7C4CF0DF0C3CF0CF0A1
:1025A000DC0E0C5C050E0D5809E2899E640E0F6E60
:1025B00008D8898E640E0F6E04D8E9D7D190FF0039
:1025C0001200106A0F50106009D0A192B10EB36EC4
:1025D000B180A1A2FED7B190102AF4D71200F95011
:1025E0003B44F92602D006D02FD05B6A020E5B6016
:1025F00038D1010C03EE10F05B50E926EF50D8B44F
:102600002ED103EE00F05B50E926EF50D8B427D16D
:102610005968010E5A6E5A52D8B421D1592A03EE84
:1026200010F05B50E926EFCF5CF003EE00F0E926F6
:10263000EF505C165A505C14D8B40ED103EE10F073
:102640005B50E9265A1CEF162DA8020C5B50400D7A
:10265000F3CFD9FFF4CFDAFF100ED926070EDA2216
:10266000080E5902F350D926000EDA22DECF1BF1F4
:102670001C6BDFCF1CF1DECF0AF0DFCF0BF0DECF1B
:102680000CF0DECF0DF003EE08F05B50E9265A5057
:10269000EF141C89D8B41C991BC15DF01CC15EF0FD
:1026A00012BBDAD003EE04F05B50E9265A50EF1467
:1026B00016E003EE04F05B50E9265A1CEF1603EE19
:1026C00012F05B50E9265A50EF14D880D8B4D89055
:1026D00003E21CB9C1D044D01CB942D0BDD003EE36
:1026E00016F05B50E9265A50EF1424E103EE12F085
:1026F0005B50E9265A1CEF161CA913D003EE12F00A
:102700005B50E9265A50EF12030E0C14030A28E01E
:102710000DC00FF059C010F05BC011F05A50A4D892
:102720009BD00DC00FF059C010F05BC011F05A5093
:102730009BD892D003EE12F05B50E9265A50EF146A
:10274000D880D8B4D89003E21CB903D009D01CB902
:1027500007D003EE16F05B50E9265A1CEF167CD02A
:10276000030E0C14010A07E0030A08E0010A08E05E
:10277000030A38E005D01CB903D034D01CB932D0DC
:1027800003EE0EF05B50E926EFCF0EF01CAD03D048
:102790005A500E1A08D01CB902D05A1C0E161CA989
:1027A00002D05A500E125A500E141C89D8B41C99DB
:1027B00003EE0EF05B50E9260EC0EFFF000E1CB9D1
:1027C000010E0BAE04D0000A1C99D8B41C890AC0B3
:1027D00014F01B901BC115F01CC116F0595098EC59
:1027E0000CF001015DC01BF15EC01CF112BB34D0C6
:1027F000D8900C32D8900C32030E0C14010A07E06A
:10280000030A08E0010A08E0030A0CE005D01CB93D
:1028100003D008D01CB906D003EE18F05B50E926AF
:102820005A50EF12D8900C32D8900C32030E0C1480
:10283000010A07E0030A08E0010A08E0030A0CE0C5
:1028400005D01CB903D008D01CB906D003EE1AF08D
:102850005B50E9265A50EF12D8905A36DCD65B2AE4
:10286000C5D6000C0101800C126E0F0E0F14136EF2
:102870000F38070B146E020A02E014662AD0080E05
:102880001102F3501024156E135207E0D89015343E
:102890001C0F1A6E13504DDD16D0020E146209D0B3
:1028A00003EE1CF0D8901534E9260A0EEE6EEF6A9E
:1028B0000AD0146608D003EE1CF0D8901534E9262F
:1028C000010EEE6EEF6A03EE16F01150E92612507B
:1028D000EF1212000A500B14FF0AD8B4120027EEB0
:1028E00010F0116A020E11602ED00F6A010E106EE8
:1028F000105227E0DECF0CF0DFCF0DF00DBE19D067
:10290000070E0D16DECF0EF0129016B912800E389B
:10291000030B0FE10A500C620CD00B500D6209D072
:102920002C9012B02C800C0E11242A6E10506EECDC
:1029300019F0060ED926000EDA220F2AD89010368A
:10294000D7D7112ACFD71200236E29B013D02C90DD
:1029500029B22C80080E22242A6E23506EEC19F026
:1029600003EE10F02250E9262350EF12050E036FFC
:10297000416AD4D02066D2D021B007D003EE16F041
:102980002250E926231CEF1608D003EE16F0225041
:10299000E926D8902330FF0AEF1621B027D02C80EB
:1029A00029B22C90080E22242A6E23506EEC19F0C6
:1029B0002C8029B22C90060E22242A6E23506EEC15
:1029C00019F02C9029B22C80080E22242A6ED8905F
:1029D00023346EEC19F02C9029B22C80060E2224A0
:1029E0002A6ED89023346EEC19F098D029B21FD0FB
:1029F0002C90080E22242A6E23506EEC19F02C9095
:102A0000060E22242A6E23506EEC19F02C90080E2C
:102A100022242A6ED89023306EEC19F02C90060EEA
:102A200022242A6ED89023306EEC19F077D0D9CFBB
:102A300027F0DACF28F02250400DF3CFD9FFF4CFA2
:102A4000DAFF130ED926070EDA22080E2102F35000
:102A5000D926000EDA220F0EDF14256E255006E06F
:102A6000050A04E00F0A02E0050A27E12C9025B2CE
:102A70002C80080E22242A6E23506EEC19F02C9024
:102A800025B22C80060E22242A6E23506EEC19F0FB
:102A90002C9025B02C80080E22242A6ED89023304A
:102AA0006EEC19F02C9025B02C80060E22242A6E94
:102AB000D89023306EEC19F02DD02C80080E2224F3
:102AC0002A6E23506EEC19F02C80080E22242A6EF8
:102AD000D89023306EEC19F0080ED95E000EDA5A49
:102AE0005F0EDF1417E0060E2114266E080E220278
:102AF000F3502624246E03EE1CF0D8902434E926EB
:102B0000010EEE6EEF6A03EE16F02250E926D89021
:102B10002330EF1227C0D9FF28C0DAFF1200F95086
:102B20003944F92602D01AD031D0606B020E6061B0
:102B3000C7D003EE10F06051E926EFCF62F003EE4C
:102B400000F0E926EF1C6215D8B4B8D05F68010E1A
:102B5000616F6153D8B4B2D05F2A010C03EE10F05C
:102B60006051E926EFCF62F003EE00F0E926EF1C9A
:102B7000621761516215D8B49ED003EE10F0605117
:102B8000E926611DEF16010112AB3AD000012DA814
:102B9000020C6051400DF3CFD9FFF4CFDAFF110ED4
:102BA000D926070EDA22080E5F02F350D926000E4E
:102BB000DA22DDCF0BF00BBC7ED00B38030B7BE1B0
:102BC000DECF0CF00D6ADECF0DF003EE08F06051A1
:102BD000E9266151EF140D88D8B40D98DFAE04D00A
:102BE000000A0D98D8B40D88100E146E1B900CC0FE
:102BF00015F00DC016F05F5098EC0CF000015BD0A2
:102C000000016051400DF3CFD9FFF4CFDAFF110E70
:102C1000D926070EDA22080E5F02F350D926000EDD
:102C2000DA22DECF63F0DECF64F0DECF65F00F0E88
:102C30006515666F6539070B656F030E64150CE04B
:102C400065C010F066C011F063C012F05FC013F0F1
:102C500060C014F0615145D9DCCF0AF0D8906433DC
:102C6000D8906433030E64150EE00AAE0CD065C034
:102C700010F066C011F063C012F05FC013F060C0C6
:102C800014F061512ED9DE50DCCF0AF0D8906433B5
:102C9000D8906433030E64150EE00AAE0CD065C004
:102CA00010F066C011F063C012F05FC013F060C096
:102CB00014F0615116D9D89061374BD7602B36D7B5
:102CC000000CF9503D44F92602D012D01FD0696B98
:102CD000020E69617DD003EE18F06951E926EF50CC
:102CE00075E06769010E686F685370E0672B010C2F
:102CF00003EE10F06951E9266851EF1464E103EE28
:102D000018F06951E9266851EF145DE02DA8020C16
:102D100003EE18F06951E926681DEF166951400D60
:102D2000F3CFD9FFF4CFDAFF100ED926070EDA223F
:102D3000080E6703F350D926000EDA22DCCF0AF022
:102D4000030ED926000EDA22DECF0BF00C6A3F0EFE
:102D5000DF140C6EDFCF0DF002EEA8F06951E9260A
:102D60006851EF140C88D8B40C980E900ABE0E80EF
:102D700003EE00F06951E9266851EF140EE00EB041
:102D80000CD00A38030B09E103EE0CF06951E92677
:102D90006851EF140C88D8B40C98010112AB07D01D
:102DA0000D38030B0F6E0F6602D0100E0D6E0DC0A6
:102DB00014F01B800BC015F00CC016F00001675119
:102DC00098EC0CF00001D89068378ED7692B80D72B
:102DD000800CF9503E44F92602D012D01FD06B6B04
:102DE000020E6B617DD003EE1AF06B51E926EF50B5
:102DF00075E06C69010E6A6F6A5370E06C2B010C10
:102E000003EE10F06B51E9266A51EF1464E103EE12
:102E10001AF06B51E9266A51EF145DE02DA8020CFF
:102E200003EE1AF06B51E9266A1DEF166B51400D47
:102E3000F3CFD9FFF4CFDAFF100ED926070EDA222E
:102E4000080E6C03F350D926000EDA22DCCF0AF00C
:102E5000050ED926000EDA22DECF0BF00C6A3F0EEB
:102E6000DF140C6EDFCF0DF002EEAAF06B51E926F5
:102E70006A51EF140C88D8B40C980E900ABE0E80DC
:102E800003EE00F06B51E9266A51EF140EE00EB02C
:102E90000CD00A38030B09E103EE0CF06B51E92664
:102EA0006A51EF140C88D8B40C98010112AB07D00A
:102EB0000D38030B0F6E0F6602D0100E0D6E0DC095
:102EC00014F01B800BC015F00CC016F000016C5103
:102ED00098EC0CF00001D8906A378ED76B2B80D716
:102EE000800C156E03EE08F01450E9261550EF140F
:102EF000D8B48DD0080E1402F3501324166E10525D
:102F000003E0020E106208D0D89016341C0F1A6E1F
:102F1000115099EC11F01AD0104C03D0030E10622E
:102F200008D0D89016341C0F1A6E1150E4EC11F032
:102F30000DD01050040A03E0060E106207D0D8909E
:102F400016341C0F1A6E115032EC12F003EE1CF006
:102F5000D8901634E926EECF18F0EECF19F01050C5
:102F6000020A0BE0010A14E0050A12E0060A2DE04D
:102F7000010A36E0050A34E048D01850191008E17B
:102F800003EE06F01450E9261550EF12D890120007
:102F900003EE16F01450E9261550EF1436E103EE57
:102FA00006F01450E9261550EF1A03EE1CF0D890E5
:102FB0001634E92618C0EEFF19C0EEFF03EE16F036
:102FC0001450E9261550EF1220D01850191008E1BE
:102FD00003EE06F01450E9261550EF12D8901200B7
:102FE00003EE06F01450E9261550EF1203EE1CF024
:102FF000D8901634E92618C0EEFF19C0EEFF03EE94
:1030000016F01450E9261550EF12D8801200105017
:10301000020A0BE0010A09E0050A07E0060A0BE0D4
:10302000010A09E0050A07E00CD003EE16F014507F
:10303000E926151CEF1603EE06F01450E926151CC0
:10304000EF16D8901200F9503C44F92601D005D073
:103050006D6B020E6D61B6D0010C03EE16F06D5172
:10306000E926EF50D8B4ACD00B68010E0A6E0A52B4
:10307000D8B4A6D00B2A03EE16F06D51E9260A50FB
:10308000EF14D8B499D06D51400DF3CFD9FFF4CFE0
:10309000DAFF100ED926070EDA22080E0B02F350C3
:1030A000D926000EDA22DCCF0CF0DCCF0EF0DCCF1C
:1030B0000DF00D38070B0F6E03EE1CF0080E6D03BC
:1030C000F3500B24D890E834E926EE06000EEF5AB0
:1030D00003EE1CF0080E6D03F3500B24D890E83477
:1030E000E926EE50EF1068E103EE00F06D51E9269D
:1030F000EF1C0A144FE00CAC19D0080ED926000EB4
:10310000DA220D38F00B0D6E0F0EDF140D26080EAF
:10311000D95E000EDA5A0FC010F00DC011F00BC0CE
:1031200012F06DC013F00A504ED846D00F50020A6C
:1031300006E00F50030A03E0060E0F6213D003EE01
:1031400016F06D51E9260A1CEF160FC010F00F0E95
:103150000D14116E126A0BC013F06DC014F00A50FA
:10316000C0DE14D00F5205E00F4C03D0040E0F62E6
:103170000DD003EE16F06D51E9260A1CEF1603EE92
:1031800006F06D51E9260A1CEF1616D0010112ABAC
:1031900013D012D003EE16F06D51E9260A1CEF167B
:1031A00003EE04F06D51E9260A50EF1203EE10F021
:1031B0006D51E9260A50EF12D8900A36000157D710
:1031C0006D2B47D7800C146E03EE06F01350E926E2
:1031D000196AEFCF18F0125005E01A6ED890183225
:1031E0001A2EFCD7196A030E18161114186212D081
:1031F0002C9011B42C80060E13242A6E14506ED815
:103200002C9011B62C80060E13242A6ED8901434FC
:1032100065D811D02C9011B02C80060E13242A6E84
:1032200014505CD82C9011B22C80060E13242A6EF8
:10323000D890143453D811380F0B116E080E1302A6
:10324000F3501224156E03EE16F01350E926141CE9
:10325000EF161050020A05E0010A1DE0050A1BE006
:1032600033D0D89015341C0F1A6E115099EC11F010
:1032700003EE1CF0D8901534E926EECF16F0EECF11
:1032800017F01650171020E003EE16F01350E92641
:103290001450EF1219D0D89015341C0F1A6E11501B
:1032A000E4EC11F003EE1CF0D8901534E926EECFD3
:1032B00016F0EECF17F01650171006E003EE16F0DA
:1032C0001350E9261450EF1203EE1CF0D890153479
:1032D000E92616C0EEFF17C0EEFF12002B6E030E9C
:1032E000EA6E2AC0E9FFD8902B50EF14D8A4D880FA
:1032F0002CA003D02B50EF1202D02B1CEF16120083
:103300000001F9503A44F92601D012D37069010E38
:103310006F6F6F53D8B40FD3702B726B27EE53F0CF
:10332000080E7003F350D926000EDA22DFCF71F0B9
:1033300071BF72857139070B716F07C36EF06F51E2
:103340006E157283D8B472936F510201A5150001F6
:103350007281D8B47291705115E0010A5FE0030ADE
:10336000D8B4A8D0010AD8B4F1D0070AD8B43AD159
:10337000010AD8B483D1030AD8B4CCD1010AD8B495
:1033800015D25FD20101399535913895349D060EDD
:103390000001716311D07251010A07E0060A05E0CD
:1033A000040A07E0060A05E007D001013581348DE3
:1033B00003D0010139853885040E0001716118D0F0
:1033C00072510FE0010A0DE0070A0BE0010A09E063
:1033D000050A0BE0010A09E0070A07E0010A05E017
:1033E00007D001013581348D03D00101398538853D
:1033F000040E0001716325D27251020A07E0050A2A
:1034000005E0040A07E0050A05E01BD20101358149
:10341000348D17D201013985388513D20101389FC7
:10342000359338973999060E0001716311D07251A6
:10343000010A07E0060A05E0040A07E0060A05E0BB
:1034400007D001013583398903D00101388F3887CE
:10345000040E0001716118D072510FE0010A0DE0F5
:10346000070A0BE0010A09E0050A0BE0010A09E07E
:10347000070A07E0010A05E007D001013583398911
:1034800003D00101388F3887040E00017163D9D150
:103490007251020A07E0050A05E0040A07E0050A7E
:1034A00005E0CFD1010135833989CBD10101388FB6
:1034B0003887C7D10101399734993899389D060E5C
:1034C0000001716311D07251010A07E0060A05E09C
:1034D000040A07E0060A05E007D001013489388DA7
:1034E00003D0010139873889040E0001716118D0B9
:1034F00072510FE0010A0DE0070A0BE0010A09E032
:10350000050A0BE0010A09E0070A07E0010A05E0E5
:1035100007D001013489388D03D0010139873889FA
:10352000040E000171638DD17251020A07E0050A91
:1035300005E0040A07E0050A05E083D101013489AA
:10354000388D7FD10101398738897BD101013991CB
:103550003497389B3993060E0001716311D0725174
:10356000010A07E0060A05E0040A07E0060A05E08A
:1035700007D001013487398303D001013981388BA9
:10358000040E0001716118D072510FE0010A0DE0C4
:10359000070A0BE0010A09E0050A0BE0010A09E04D
:1035A000070A07E0010A05E007D0010134873983E3
:1035B00003D001013981388B040E0001716341D1C0
:1035C0007251020A07E0050A05E0040A07E0050A4D
:1035D00005E037D101013487398333D101013981C5
:1035E000388B2FD101013797369F369D3795060EC0
:1035F0000001716311D07251010A07E0060A05E06B
:10360000040A07E0060A05E007D00101368F378576
:1036100003D001013787368D040E0001716118D087
:1036200072510FE0010A0DE0070A0BE0010A09E000
:10363000050A0BE0010A09E0070A07E0010A05E0B4
:1036400007D00101368F378503D001013787368DCA
:10365000040E00017163F5D07251020A07E0050AF9
:1036600005E0040A07E0050A05E0EBD00101368F0A
:103670003785E7D001013787368DE3D00101379DCB
:10368000369B3699379F060E0001716311D0725137
:10369000010A07E0060A05E0040A07E0060A05E059
:1036A00007D00101368B378F03D00101378D368962
:1036B000040E0001716118D072510FE0010A0DE093
:1036C000070A0BE0010A09E0050A0BE0010A09E01C
:1036D000070A07E0010A05E007D00101368B378FA2
:1036E00003D00101378D3689040E00017163A9D022
:1036F0007251020A07E0050A05E0040A07E0050A1C
:1037000005E09FD00101368B378F9BD00101378DAB
:10371000368997D001013793369536933791060E47
:103720000001716311D07251010A07E0060A05E039
:10373000040A07E0060A05E007D001013685378153
:1037400003D0010137833683040E0001716118D064
:1037500072510FE0010A0DE0070A0BE0010A09E0CF
:10376000050A0BE0010A09E0070A07E0010A05E083
:1037700007D001013685378103D0010137833683B5
:10378000040E000171635DD07251020A07E0050A60
:1037900005E0040A07E0050A05E053D0010136857B
:1037A00037814FD00101378336834BD001013799E0
:1037B00036973691379B060E0001716311D0725116
:1037C000010A07E0060A05E0040A07E0060A05E028
:1037D00007D001013687378B03D001013789368145
:1037E000040E0001716118D072510FE0010A0DE062
:1037F000070A0BE0010A09E0050A0BE0010A09E0EB
:10380000070A07E0010A05E007D001013687378B78
:1038100003D0010137893681040E0001716311D094
:103820007251020A07E0050A05E0040A07E0050AEA
:1038300005E007D001013687378B03D001013789B6
:10384000368134C174F00001745101013A6302D031
:1038500014A90FD0000174A7899674B7898674A93A
:10386000899874B9898874AD899C74BD898C74C039
:103870003AF135C174F00001745101013B6302D08B
:1038800014A90AD08BCF75F0030E00017415756F63
:1038900075C08BFF74C03BF136C174F000017451E8
:1038A00001013C6302D014A909D08CCF75F000014E
:1038B0007451756F75C08CFF74C03CF137C174F0E2
:1038C0000001745101013D6302D014A909D08DCFCC
:1038D00075F000017451756F75C08DFF74C03DF1B6
:1038E00038C174F00001745101013E6302D014A983
:1038F0000AD08ECF75F0FC0E00017415756F75C07F
:103900008EFF74C03EF139C174F0000174510101A1
:103910003F6302D014A90AD08FCF75F01F0E0001AB
:103920007415756F75C08FFF74C03FF10101010CF4
:10393000D8906F37EED40101800C0A6A06C30BF0F1
:10394000001D0B1614510B1A03EE00F00A50E92665
:10395000EFB005D00BA08B960BB08B8607D003EE93
:1039600002F00A50E926EF9082B6EF8003EE00F0F5
:103970000A50E926EFB205D00BA28B940BB28B84D0
:1039800007D003EE02F00A50E926EF9282B4EF82EC
:1039900003EE00F00A50E926EFB405D00BA48B9A91
:1039A0000BB48B8A07D003EE02F00A50E926EF949D
:1039B00082BAEF8403EE00F00A50E926EFB605D094
:1039C0000BA68B980BB68B8807D003EE02F00A503B
:1039D000E926EF9682B8EF8603EE00F00A50E9265A
:1039E000EFB805D00BA88A980BB88A8807D003EEE9
:1039F00002F00A50E926EF9881B8EF8803EE00F054
:103A00000A50E926EFBA05D00BAA8A960BBA8A8625
:103A100007D003EE02F00A50E926EF9A81B6EF8A4A
:103A200003EE00F00A50E926EFBC05D00BAC8A94F7
:103A30000BBC8A8407D003EE02F00A50E926EF9C03
:103A400081B4EF8C03EE00F00A50E926EFBE05D0FA
:103A50000BAE8A920BBE8A8207D003EE02F00A50A8
:103A6000E926EF9E81B2EF8E03EE00F00A50E926C0
:103A7000EF500B1603EE02F00A50E9260B50EF1A36
:103A80001200F9503F44F92602D0E5D058D1800EFB
:103A9000366E2C9A766B200E766153D1080E760323
:103AA000F350900F776F070E786B782377C0D9FFAC
:103AB00078C0DAFFDFAE43D1040ED924E16E000EE8
:103AC000DA20E26E2C98E6CF0BF0E7CF0CF00D6A0F
:103AD000E7BC0D2A0E90E7B80E80DFB802D0E7AE43
:103AE0003ED0DFA803D0010113BF05D0DFB835D029
:103AF000010113BF32D00C980BC00FF00CC010F0B6
:103B000015C111F016C112F00D5000019EEC0FF01E
:103B100014C00AF00ABE21D002EE85F000017651F1
:103B2000E926EF9C0AB00CD002EE85F0E926EF9A68
:103B30000AB0EF8A02EE85F0E926EF900AB0EF8036
:103B400002EE85F07651E926EF900AB0EF800EA0E4
:103B500004D002EE85F0E926EF8C000105D002EEDC
:103B600085F07651E926EF80060ED924E16E000E2D
:103B7000DA20E26EE6CF0BF0E7CF0CF00D6AE7BC7F
:103B80000D2A0E90E7B80E80DFB602D0E7AE35D032
:103B9000DFA603D0010113BF05D0DFB62CD0010191
:103BA00013BF29D00C980BC00FF00CC010F015C13A
:103BB00011F016C112F00D5000019EEC0FF014C070
:103BC0000AF00ABE18D002EE85F000017651E9260F
:103BD000EFA004D002EE85F0E926EF8A02EE85F030
:103BE0007651E926EF920AB0EF820EA004D002EEE1
:103BF00085F0E926EF8C000105D002EE85F07651C4
:103C0000E926EF820E92DFBC0E822CBA06D07651E6
:103C10009AD82C98D8B02C8809D002EE85F076512D
:103C2000E926EF9802EE85F0E926EF9602EE85F0A0
:103C30007651E926EFB62C8A0EB22C9A2CA87ED0AB
:103C4000D9CFE1FFDACFE2FFE4BE05D002EE85F086
:103C5000E926EFB873D02DA8010C77C0D9FF78C042
:103C6000DAFFD9CFE1FFDACFE2FF070EE4140FE06D
:103C7000010A11E0030A13E0010A15E0070A17E040
:103C8000010A19E0030A1CE0010A1FE022D0010E1C
:103C90000A6E0B6A1ED0050E0A6E0B6A1AD00A0E47
:103CA0000A6E0B6A16D0320E0A6E0B6A12D0640EC0
:103CB0000A6E0B6A0ED0F40E0A6E010E0B6E09D05E
:103CC000E80E0A6E030E0B6E04D0880E0A6E130EF9
:103CD0000B6EE738E8461F0B0F0B0C6E0C2A0A50D0
:103CE0000C02F3CF0DF0F4CF0EF00F6A0B500C0264
:103CF000F3500E26F4500F220CAE04D00A500E5E84
:103D00000B500F5A0BAE02D00C500F5E0D500E1020
:103D10000F1012E003EE3CF0030E7603F350E92699
:103D20000DC0EEFF0EC0EEFF0FC0EEFF02EE85F0FD
:103D30007651E926EF8802D07651BBD8020C762B5B
:103D4000AAD6366A800C0F6E1190080E0F02F3503F
:103D5000900FE16E070EE26AE22202EE85F00F504C
:103D6000E926D890E73006E3EFB002D0EFA206D004
:103D7000118004D0EFA002D0EFB21180D890E730CC
:103D8000030B106E105007E0010A1DE0030A33E038
:103D9000010A41E05BD011A013D0EFBC07D011B0F5
:103DA00003D0EFB403D007D0EFB405D0EF86EF8493
:103DB000EF9CD8801200EFB649D0EF86D880120071
:103DC000EF96EF9443D011B013D0EFBC07D011B0F1
:103DD00003D0EFB403D007D0EFB405D0EF86EF9453
:103DE000EF9CD8801200EFB631D0EF86D880120059
:103DF000EF96EF842BD0EFBC07D011B003D0EFB417
:103E000003D024D0EFB422D011A0EF9411B0EF84EE
:103E1000EF9CD880120011A017D0EFBA02D0D89032
:103E20001200EFBC07D011B003D0EFB403D007D01D
:103E3000EFB405D0EF86EF84EF9CD8801200EFB688
:103E400005D0EF86D8801200EF96EF94D89012003C
:103E5000F9504044F92602D006D024D0796B200EC8
:103E6000796126D0010C02EE85F07951E926EFA8A0
:103E70001DD003EE3CF0030E7903F350E926EE0665
:103E8000000EEE5AEF5A03EE3CF0030E7903F350A6
:103E9000E926EE50EE10EF1009E102EE85F07951BF
:103EA000E926EF982DA8020C795103D8792BD7D7A2
:103EB000800C106E080E1002F350900FE16E070E8A
:103EC000E26AE222E7AA12D0020EE126000EE22206
:103ED000E6CF11F0126AE7CF12F011C013F012C052
:103EE00014F001011CEC0FF0000118D0020EE126C5
:103EF000000EE222E6CF11F0126A0F0EE714126EE6
:103F00001288E7CF13F013C014F01B8011C015F016
:103F100012C016F0000E98EC0CF00001120009A37C
:103F200012000101032B032B04EE00F00351E926DC
:103F30007C0EEF625CD0032B04EE00F00351E92607
:103F4000EFCF0CF0032B032B04EE00F00351E92616
:103F5000EFCF0BF0032B04EE00F00351E926D890CD
:103F6000EF340A6E0B340B320A320A5002016B63D3
:103F700004D00B506C6301D00BD0010114A307D007
:103F80000F0E0A6204D0270E0B6201D001D012007E
:103F90000101032B032BFC0E0C14200A0BE0080A72
:103FA00009E0040A11E04C0A19E0080A17E00C0ABB
:103FB0001AE01DD00CC00DF00AC00EF00BC00FF0BF
:103FC00017D8010ED8D913D00CC00DF00AC00EF0CE
:103FD0000BC00FF00DD8010ECED909D005D9400E77
:103FE0000101C9D904D000D9400E0101C4D9120081
:103FF00012EE2BF00E0EE66EE70EE66E0E0EE66E7D
:104000007C0EE66E0DC0E6FFE66AD8900E360F36DF
:10401000D8900E320FC0E6FF0EC0E6FFE66A166AC1
:1040200004EE00F00351E926EFCF14F014C013F0B2
:1040300013380F0B136E032B04EE00F00351E92627
:10404000EFCF15F015C012F0129E14B0128E17901B
:10405000125013100AE1040E126E136AE96E070E75
:104060001324EA6EEFCF16F01780135003E1050E0C
:10407000126412D0135010E1090E12600DD0060E1A
:10408000125E000E135A1250E96E070E1324EA6EE8
:10409000EFCF16F0178093D0100E126202D0135299
:1040A00005E0110E12620FD013660DD00C0E125ED9
:1040B000000E135A1250E96E070E1324EA6EEFCF6A
:1040C00016F017807CD01B0E126202D0135205E04E
:1040D0001C0E12620FD013660DD0150E125E000E6C
:1040E000135A1250E96E070E1324EA6EEFCF16F042
:1040F000178065D06F0E126214D0136612D0660E50
:10410000125E000E135A1250E96E070E1324EA6E67
:10411000EFCF16F014A303D0169214B116821780B5
:104120004ED0135003E16F0E126413D0135011E1FF
:10413000730E12600ED0670E125E000E135A900EB0
:104140001224E96E080E1320EA6EEFCF16F01780E6
:1041500036D0740E12620ED013660CD0660E125E4C
:10416000000E135A1250E96E070E1324EA6EEFCFB9
:1041700016F025D0135002E112AE12D0135010E108
:1041800012480ED0800E125E000E135A100E12242A
:10419000E96E070E1320EA6EEFCF16F017800FD0EE
:1041A00013520DE0020E13600AD01306900E122473
:1041B000E96E070E1320EA6EEFCF16F01780149207
:1041C00016BE148214C0E6FF15C0E6FF7F0E16145B
:1041D000E66EE66AE66A17A005D0050E0201036FD7
:1041E000416A0101138312001190010114AD0ED038
:1041F0000C0E02017C150C0AD8A41200030E7C15CB
:10420000106E7DC20FF07EC20DF0010114AB1DD007
:1042100004EE00F00351E926EFCF10F0032B04EE7B
:1042200000F00351E926EFCF0FF00F9E10B00F8E74
:10423000032B04EE00F00351E926EFCF0DF00D9EA5
:1042400010B20D8E10380F0B106E10502FE1200E93
:104250000F602CD0100E0F6202D0105205E0110E2C
:104260000F620ED010660CD00C0E0F5E000E105AAE
:104270000F50E96E070E1024EA6E0DC0EFFF6AD0F2
:104280001B0E0F6202D0105205E01C0E0F6262D0AE
:10429000106660D0150E0F5E000E105A0F50E96EBA
:1042A000070E1024EA6E0DC0EFFF54D06F0E0F62A0
:1042B00013D0106611D0660E0F5E000E105A0F500C
:1042C000E96E070E1024EA6E800E0D10EF6E149149
:1042D0000DB2148111803ED0740E0F620FD01066A3
:1042E0000DD0660E0F5E000E105A0F50E96E070ECD
:1042F0001024EA6E0DC0EFFF11802CD0105002E1A7
:104300000FAE14D0106612D0800E0F5E000E105A41
:10431000100E0F24E96E070E1020EA6E0DC0EFFF9D
:10432000100E0F26000E1022118014D0105211E032
:10433000020E10600ED01006900E0F24E96E070ECC
:104340001020EA6E0DC0EFFF900E0F26000E102217
:1043500001D012000FC012F010C013F00D505BD846
:1043600011A004D06FD9C8D901010EDA050E0201DF
:10437000036F416A12000D6E0751E96E050E0825A4
:10438000EA6E040EEF6EA8EC10F00751E96E050E10
:104390000825EA6EB40EEF6EA8EC10F00751E96E36
:1043A000050E0825EA6E6F0EEF6EA8EC10F00751AF
:1043B000E96E050E0825EA6E0DC0EFFFA8EC10F0BF
:1043C0000551075D0E6E065108590F6E0FAE02D0F3
:1043D000020E0F260FBE06D0E10E0E5C010E0F5826
:1043E000D8B02D981200032B04EE00F00351E926FB
:1043F0006F0EEF6204D013A302D01393376A12003A
:104400007FB2FED715C062FF16C063FF7F9E7F9C00
:104410007F8061501200146E12C015F013C016F0A8
:10442000EFDF14181CE07FB2FED714C061FF12C08A
:1044300062FF13C063FF7F9E7F9C7F84F29E550EB8
:104440007E6EAA0E7E6E7F82F28E7F9412C015F071
:1044500013C016F0D5DF141802E0D8901200D880EF
:1044600012007FCFF6FF7FCFF7FFF86A7F8E7F9C29
:104470000800F5501200F00ED36EC00E9B6E800E39
:10448000806E270E926E200E816EDF0E936E826A12
:10449000BC0E946E836A956A846A966A856A020E77
:1044A000976E866A986A570E256F246B236B010EF0
:1044B000C26E300EC16EBE0EC06E200EAC6E900E7F
:1044C000AB6E100E656E3B0EAF6EF26A800EF16E33
:1044D000F06A9D6AA06A9F6AA26AD59ED66A340E67
:1044E000CD6E9E909D90CE0ECA6ECA949E929D9265
:1044F000300EB16E0FEE15F0ED6AEA50FDE1E950B5
:10450000FBE1EF6A0B0EC26EC2B2FED7C4CF0BF056
:10451000C3CF0AF0DC0E0A5C050E0B580BE2899E35
:10452000640E0F6EE1EC12F0898E640E0F6EE1ECFA
:1045300012F0E8D70AC021F10BC022F10D019283DD
:10454000110EC26E0A0E0F6EE1EC12F0C2820F0164
:10455000C2B2FED7C4CF0DF0C3CF0CF00F0E0D6466
:1045600002D00C6A0D6AA10E0C5C0F0E0D5802E30E
:10457000D8801200D890120007EE00F00A6A0B6A89
:104580000AC015F00BC016F03BDFEE6E0A2A000ED3
:104590000B229C0E0A5C010E0B58F2E399C800F244
:1045A0009AC801F29BC802F23F0E070104150201EE
:1045B0006C6F05C76BF27F8E7F9CF66AF76A200EE0
:1045C000F86E0EEE40F0080E126E0900F5CFEEFF09
:1045D000122EFBD745CE48FE130EC26E0101C2B2A9
:1045E000FED7C4CF11F0C3CF10F00F0E116402D06C
:1045F000106A116A149F149D149BDC0E105C050E4A
:10460000115802E2148B17D0DD0E105C050E115804
:1046100007E3A40E105C060E115802E2148D0BD0B5
:10462000FD0E105C080E115806E3280E105C0A0EF1
:104630001158D8A0148F14BD04D014BF02D014ABED
:10464000148B120027EE12F0156A0301020E15609A
:1046500027D0010E146E03EE14F01550E926EF6A10
:1046600003EE00F0E926EF6ADFAC07D003EE00F0BE
:104670001550E9261450EF1209D0DCAE06D003EE37
:1046800014F01550E9261450EF12DD50D89014366E
:10469000080ED926000EDA221466E6D7152AD6D7D8
:1046A00000A1949600B1948600A3949400B39484DE
:1046B00000A5949A00B5948A00A7949800B79488AE
:1046C00000A9939800B9938800AB939600BB93869A
:1046D00000AD939400BD938400AF939200BF93828A
:1046E0000EC72DF101012E6B040E166ED8902D37DA
:1046F0002E37162EFBD7120027EE11F0136A030196
:10470000020E13603ED0010E156E146ADFCF16F054
:10471000020ED926000EDA22DFCF17F01738070B6A
:10472000176E16BC04D0040A02E015501412D8907B
:104730001536060ED926000EDA221566E7D70701D0
:1047400009A11CD0900E1324E96E080EEA6AEA2231
:10475000EFCF12F003EE08F01350E92614501214B4
:10476000EF6E03EE00F01350E926EF1C126E03EE1D
:1047700010F01350E92614501214EF6E132A03019F
:10478000BFD7004908691200016B126A100E12604F
:104790000CD0080E1202F350100FD96E070EDA6A11
:1047A000DA22DF500127122AF1D7040E02016B032F
:1047B000F350010101273F0E011701C106F7120056
:1047C0000A6A01510A600BD0A192B368B26AB18043
:1047D000A1A2FED7B19012B502D00A2AF2D71200D8
:0200000400F00A
:100000000B571C00270F00E0009F00000000640059
:100010000020430000000000012043000000000019
:100020000220430000000000032043000000000005
:1000300004204300000000000520430000000000F1
:1000400006204300000000000720430000000000DD
:100050000800030000000000090003000000000089
:100060000A000300000000000B0003000000000075
:100070000C000300000000000D0003000000000061
:100080000E000300000000000F000300000000004D
:100090000000000000000000000000000000000060
:1000A0000000000000000000000000000000000050
:1000B0000000000000000000000000000000000040
:1000C0000000000000000000000000000000000030
:1000D0000000000000000000000000000000000020
:1000E0000000000000000000000000000000000010
:1000F0000000000000000000000000000000000000
:1001000000000000000000000000000000000000EF
:1001100000000000000000000000000000000000DF
:1001200000000000000000000000000000000000CF
:1001300000000000000000000000000000000000BF
:1001400000000000000000000000000000000000AF
:10015000000000000000000000000000000000009F
:10016000000000000000000000000000000000008F
:10017000000000000000000000000000000000007F
:10018000000000000000000000000000000000006F
:0C01900000000000000000000000000063
:020000040000FA
:0400000000EF02F01B
:020000040030CA
:0E000000B6383300FE897FFF8FC10FE00F403E
:00000001FF
